:03000000020030CB
:03000300020F8960
:03000B00020FD908
:03001300020FA534
:03001B0002102EA2
:10003000C287C28612099C60030200D1120C61754E
:1000400087807581C078087978B83003020063B87A
:100050003103020063B83203020063B833030200C5
:1000600063760008D9E3753AFF7570FF7562FF7516
:1000700063FF7564FF120C221209B960381209E897
:1000800060331208FE602E853B2F1209B960267876
:100090009DE6FC08E6FB8C348B35120A386016307E
:1000A000B719789AE6FC08E6FB8C348B35120A38CF
:1000B00060030200BB753A887570FF20B503754672
:1000C00014754A03754FAE75509E1209AFC2970161
:1000D000CF204B02D28775C83475891175CAFA755D
:1000E000CBFF758805759850758780E5502476F5A7
:1000F0008AE54F3400F58CD28C7581C075B80375D4
:10010000A88F30490CE5254551F525E5264552F5E2
:1001100026852521852622D245754C00754B001277
:100120000C22E53AB4FF03020150E54E6003D54EC0
:100130001CE54A6018154A754E0A120C6A75470389
:10014000754803754903304B04D248C24B02015035
:100150001205CCE574B404030205831206F5120EF1
:10016000BF7858120F2130460B755400120C61C233
:10017000460201DE7858120F2130460B75540012EA
:100180000C61C2460201DE7858120F2130460B7511
:100190005400120C61C2460201DE78687600120F2C
:1001A0005730460B755400120C61C2460201DE1234
:1001B0000EF37868120F5730460B755400120C611D
:1001C000C2460201DE120EF37868120F5730460B5A
:1001D000755400120C61C2460201DE120EF3E554A2
:1001E000B5530685532B0201EC8554538560363098
:1001F000B7097574007575000201FE75360EE57459
:10020000B404030205751209B97009753A8875704E
:10021000FF02057578A386410886400808088644D1
:10022000088643789F863F78A0866178AF8652081B
:100230008651E53AB4FF0302029E789DE6FC08E68B
:10024000FB8C348B35120A3860C1E52FB4FE0302F3
:100250000263B4FF03020263789AE6FC08E6FB8CB3
:10026000348B35E53AB4CC1E7892E6F52608E6F5EF
:10027000257896E6F55608E6F55585252C85262D34
:10028000753C0E02057575250075260075550075BF
:100290005600752C00752D00753C0F020575AC34A9
:1002A000AB35120A387002410BE52BA2E79243549A
:1002B0000FF52BE574B401068557360202C0707A3B
:1002C0007891E6B40E17E52FB4FF12752500752658
:1002D00000755500755600753C0F020315E6F53C98
:1002E0007892E6F52608E6F5257896E6F55608E6CE
:1002F000F555E53CB40E03020315304918E52545D4
:1003000051F525E5264552F526E5554551F555E5C6
:10031000564552F55685252C85262D053778A0E6BD
:10032000C537B53700C53750030205757891E654D7
:100330000FB40D06753700020525E5746012B4028E
:100340001275430075440075400075410002036258
:100350000203FDB403FA7543FF7544FF7540FF7552
:1003600041FF752500752600E575B4010675260860
:100370000203F7B402067526800203F7B40306757C
:1003800026100203F7B404067525040203F7B4052A
:10039000067526010203F7B406067525200203F749
:1003A000B407067526040203F7B40806752508028B
:1003B00003F7B409067526200203F7B40A0675256B
:1003C000400203F7B40B067525100203F7B40C06C0
:1003D0007525020203F7B40D067526400203F7B433
:1003E0000E067526020203F7B40F06752580020378
:1003F000F7B41003752501852555852656E5366029
:100400003DB40E06753BFE020431B40F06753BFF8A
:10041000020431E53FB53614789EE6B4FF0808E6DD
:10042000B4FF0302042E753BFD0204314010753BFE
:1004300001D244E536B53C03020575020525C244E8
:10044000E52B602FB40E06753BFE020453B40F0E6D
:10045000753BFF753803E52BB53CE0020575E53FBC
:10046000B52B00400E753B01753803E52BB53C0CF0
:1004700002057530432B753803020575789EE6B486
:10048000FF0808E6B4FF03020525E53FB52B0C2065
:1004900043033049A3753BFD020525753B01020569
:1004A00025E5386005D53890C24330493FE53CB476
:1004B0000E004005C2490204EC789EE6B4FF1C0819
:1004C000E6B4FF17304C04C24CD24E304E1EE53C11
:1004D000B40152753700C24E02057520490302046B
:1004E000EC753BFDE53CB53F3C020575E53CB40EC3
:1004F00003020513B40F03020513E52FB4FD0274C4
:100500000178A086F028F8E625F0C537B53700C594
:100510003740621209237002410BAC34AB35120A2A
:10052000387002410BE53BB4FD05789E020541B4ED
:10053000FF05789C020541B4FE05789C02054178D0
:100540009AE6FC08E6FB8C348B35120A38700241BF
:100550000B7892E6452CF52C08E6452DF52D853BCC
:100560002F7891E6B53C0302056D7537007891E66A
:10057000B53F02C249752B007536003042FDC242BC
:100580001206F54387013047FA752300752400757C
:100590002500752600755500755600753E00753DA1
:1005A00000753AEE7570FF120C7A753C0F752FFFCF
:1005B000753800C243754E0A754A03C28C858C4F4C
:1005C000858A50C2471209AFC297A183E54CB40790
:1005D00000400302066130B706757400020661E54B
:1005E00074702A787676D30876020876000876004A
:1005F0001207B91207E560697876E6B4D3CE08E64B
:10060000B402C908E6B480C4757404A1CCB4045122
:10061000787676D30876020876800876001207B9D5
:100620001207E5603C7876E6B4D3A108E6B402325E
:1006300008E6B4812608E6547FC0E075F010A4C532
:10064000F0787A7910120BD9787676D3087612087A
:10065000768108D0E0F61207B9A1CCB48FFB75748F
:100660000022B412F408E6B482EF08E6547FC0E03A
:1006700075F010A4C5F07910787AC282120C047556
:100680006504E56570FCD282787A7910D0E0C0E02C
:1006900075F010A4C5F01206B9400675F083020685
:1006A000A475F084787676D308761208A6F008D080
:1006B000E0F678761207B9A1CCB2E2120A6BC33326
:1006C000C0E044A0120A8BE5F0120A8B120A6BD02C
:1006D000E044A1120A8B120B1CF5F0E6B5F01408E9
:1006E000B901030206E9120B04D9EB120B10120A2E
:1006F0007BC322D322787676020876020876000839
:1007000076001207B91207E560187876E6B402128F
:1007100008E6B4020D0808E6B45F0876FF787612A2
:1007200007B92218E6B40508120C3208A631E11DFB
:10073000B40608120C4208A632E11DB40708120CD8
:100740005208A633E11DB408150574E574B401031D
:10075000757501B4040375740008A674E11DB4092D
:100760004B0575E574B40122E575B41000400675BB
:1007700075010207A7B40E00502D853FF005F0B5B6
:10078000F000402375750E0207A7B4020DE575B49D
:10079000110040137575000207A7B4030AE575B48C
:1007A0001100400375750008A675E11DB40A0385A4
:1007B000755708E6F9E7F6E11D7876E4869926088C
:1007C0003099FDC29986F0869926083099FDC29924
:1007D000869926083099FDC299D5F0F4F59908302C
:1007E00099FDC2992275650A7876209806E56560BC
:1007F00064E1EAC298E599B40203020806B4E4038E
:10080000020806B4D3E4F608756504209806E56589
:100810006043010BC298AA99A699087565042098AF
:1008200006E5656030011EC298A69908DAED756587
:1008300004209806E565601D0131C298A699787775
:10084000E62402F5F07876E42608D5F0FB86F0B5CC
:10085000F00374FF22740022789786F008E6120BEA
:10086000BAF91414FA789786F008E67890120BD942
:100870007890E4FBFCEB26FB74003CFC08DAF6EB1A
:1008800086F0B5F00A08EC86F0B5F00374FF22E4B8
:1008900022789386F008E6120BBAF91414FA7893CA
:1008A00086F008E67890120BD97890E4FBFCEB26F2
:1008B000FB74003CFC08DAF6EB86F0B5F00A08ECB5
:1008C00086F0B5F00374FF22E4228BF0EC120BBA31
:1008D000F91414FA8BF008EC7890120BD97890E4A4
:1008E000FBFCEB26FB74003CFC08DAF6EB86F0B56B
:1008F000F00A08EC86F0B5F00374FF22E4221158E8
:10090000605C119160587890E61414141428F8E68D
:10091000FB08E6FC11CA60467890E614141428F827
:10092000E6F53B1209B96036115860321191602E1C
:100930007890E61414141428F8E6FB08E6FC789086
:10094000E614141475F00384FA7891E6C533B533D0
:1009500000C533500E08E6FB08E6FC08DAED753BEF
:10096000FEE42211CA60F77890E614141475F003BF
:1009700084FA08860308860408860508E532B5036C
:1009800011E531B504118D3BDA0302099950E402F7
:10099000099950F202099950ED74FF227821E4265A
:1009A00008B839FBF5F0E6B5F00374FF22E42278CD
:1009B00021E42608B839FBF6227890792674007570
:1009C000F000120BD97A247890E4FBFCEB26FB7440
:1009D000003CFC08DAF6EB86F0B5F00A08EC86F08D
:1009E000B5F00374FF22E4227895E6F908E6FAE907
:1009F00014B4FF011A14B4FF011AF9E4FBFC9000CF
:100A0000008582F0E583120BBA2BFB74003CFCA33B
:100A1000D9EFEA60031A41018582F0E583120BBA2F
:100A20008BF0B5F011A38582F0E583120BBA8CF040
:100A3000B5F00374FF22E422EB8CF0120BBAF9FA42
:100A40007890EB8CF0120BD97890E4FCFB1A1AEB3F
:100A500026FB74003CFC08DAF6EB86F0B5F00A08D9
:100A6000EC86F0B5F00374FF22E422D2800000D2BD
:100A7000810000C2800000C2810022C2810000C249
:100A8000800000D2810000D28000223392800000DA
:100A9000D2810000C28100003392800000D2810028
:100AA00000C28100003392800000D2810000C28128
:100AB00000003392800000D2810000C28100003328
:100AC00092800000D2810000C28100003392800039
:100AD00000D2810000C28100003392800000D281E8
:100AE0000000C28100003392800000D2810000C269
:100AF00081000033D2800000D2810000A28000007B
:100B0000C2810022C2800000D2810000C281002286
:100B1000D2800000D2810000C2810022D280000079
:100B20000000D28100000000A2800000000033C25B
:100B30008100000000D28100000000A280000000BF
:100B40000033C28100000000D28100000000A280BA
:100B50000000000033C28100000000D281000000CC
:100B600000A2800000000033C28100000000D2819A
:100B700000000000A2800000000033C281000000DD
:100B800000D28100000000A2800000000033C2817A
:100B900000000000D28100000000A28000000000E0
:100BA00033C28100000000D28100000000A280005A
:100BB00000000033C28100000022B2E2516BC33357
:100BC000C0E044A0518BE5F0518B516BD0E044A1C3
:100BD000518B711C7110517B22B2E2516BC333C037
:100BE000E044A0518BE5F0518B516BD0E044A15112
:100BF0008B711CF608B90103020BFD7104D9F27167
:100C000010517B22B2E2C33344A0516B518B50058B
:100C1000517B00810AE5F0518BE6518B08D9FA51DE
:100C20007B22E5302401D4F53024A0500375300038
:100C3000502EE5312401D4F53124A0500375310044
:100C4000501EE5322401D4F53224DC500375320005
:100C5000500EE5332401D4F53324F95003753300E5
:100C600022C2967B1FDBFED29622753AFF7570FF7B
:100C70007562FF7563FF7564FF228531628532639B
:100C800085336422E5F030E00375700330E10375CD
:100C9000700430E20375700130E30375700230E4D4
:100CA0000375700530E50375700622E5F030E0034A
:100CB00075700530E10375700230E2037570033022
:100CC000E30375700430E40375700130E50375705B
:100CD0000622E521B52303020CF35523F5236521F4
:100CE000FA7B00D3EB13400BFB5A60F84523F52346
:100CF000020D13E522B52405C245020D135524F556
:100D0000246522FA7B00D3EB134008FB5A60F845B8
:100D100024F52422E523F4F5A000C293000000D2BC
:100D200093E524F4F5A000C294000000D294C29090
:100D300075A0FFE4A22392E2A21A92E3A22292E01B
:100D4000A21E92E1A22692E4A21F92E5F53DE4A242
:100D50002492E4A21D92E1A22592E2A21992E3A2BA
:100D60002192E0A21892E5F53EE543A2E292F3A2B9
:100D7000E692F1A2E792F5E544A2E292F0A2E392B4
:100D8000F2A2E692F4E5F0553D543FF53DE540A270
:100D9000E092F5A2E192F3A2E592F1E541A2E1929F
:100DA000F0A2E492F4A2E592F2E53EF455F0543F4D
:100DB000F53E22D28600E5A0C286543F553D6036FE
:100DC000F5F0E5476003D5473075230075240075BD
:100DD0002500752600755500755600753D00753C5B
:100DE0000F753ACC9184917A754E0A752FFE75383D
:100DF00000C243020DF975470322C295D295C291F4
:100E0000000000E5A0F5F0D29120E611204D04D2BB
:100E10004CD24DE53CB53F0AC249020E24C24D02F8
:100E20000E24D249E5F0F4553E543F603BF5F0E521
:100E3000486003D548357523007524007525007575
:100E40002600755500755600753E00753D00753CD1
:100E50000F753ABB91AB917AD24B754E0A752FFF45
:100E6000753800C243020E6B75480322C295D295B5
:100E7000C291000000E5A0D291F4553E543F603B82
:100E8000F5F0E5496003D5493575230075240075F3
:100E90002500752600755500755600753E00753D98
:100EA00000753C0F753ABB91AB917AD24B754E0AE7
:100EB000752FFF753800C243020EBE75490322E547
:100EC0003C540F7858F63043067858E64480F630A4
:100ED00044067858E64440F6E53AB4FF03020EE6CD
:100EE0007858E64420F6E478587B072608DBFC783F
:100EF0005FF622E47B0778682608DBFCF5F0786F64
:100F0000E6B5F01004F678688654760008866076B8
:100F100000020F20786876007554007560009161BA
:100F2000227A08E67B04139284000000C28379329F
:100F3000308505D9FB020F52139284000000D28342
:100F40007932208505D9FB020F52DBDA08DAD4D2D8
:100F50008422D246D284227A087B04C2837932303A
:100F60008505D9FB020F86000000A28413D2837985
:100F700032208505D9FB020F86000000A28413DB16
:100F8000DAF608DAD422D24622D24B753AAA757024
:100F9000FF917A754E0A752FFF7523FF7524FF7533
:100FA0003800C24332C0E0C0F0C0D0C082C083D29B
:100FB000D3C2D430450291D2304B02C287B11475EE
:100FC0008BC0758DFCD28E754D00054BC28BD083C6
:100FD000D082D0D0D0F0D0E032758A9E758CAEC071
:100FE000E0C0F0C0D0C082C083054CE54CB4041C06
:100FF00030490CE5554551F555E5564552F55685B0
:101000005521855622D245D242021023B40814E558
:101010004BB43000400BC247D24AC292D292021067
:1010200023D247D083D082D0D0D0F0D0E032758B9D
:10103000C0758DFCC0E0C0F0C0D0C082C083D2D3E8
:10104000D2D4B2B6E56560021565054DE54DB40133
:1010500008120DFAD2900210C0B4020B304B02C23B
:1010600087120D140210C0E53AB4FF06204803129F
:101070000DB3120E6CD290C28E304A44C24AC28C5A
:10108000858C4F858A50C2481209AFC2977B00DB1E
:10109000FE75230075240075250075260075550022
:1010A000755600753E00753D00753C0F753A997593
:1010B00070FF120C7A754E0A752FFF753800C24307
:0B10C000D083D082D0D0D0F0D0E0323E
:00000001FF
